:200000008088944CB4DC24C0849078786C946CD42040D8B4302C28C0A084704C78C0807404
:2000200030A45440BCB47C3850D8D44C2C78808870908084A870BC9884B4482084F0582C38
:20004000B8B4746848687894487098983CE47428B4BC6C8C406094BC2C40E8B87074584018
:20006000AC886080D0A0A850788868809844EC446468A8B44430CC6C7C9C245C88ECA83058
:2000800060A0649C3064946C9CD890885454A03C787094C47820A4585458C07424A4D0541C
:2000A0005C689C98B8608090A8642878D4B47880788878688C7090D870945C648C74484064
:2000C000D8A8443C90CC5C6CA060C8A4684C9CA4A434A8D478A4603C54D07858B87C7C608C
:2000E000887058749454B0903C788C789054608CA48C7458A09074CC60A094189898B06430
:2001000024D8B8606870786C2CB88C7C589088A43078B4745C946898488C9C5C80C04C54A3
:20012000C460706888C0AC505CA09058B05C68B4A85834BC687CB82C749C74A08478448CCB
:20014000B09C4C5C5CB8A03C6CB45C946878BC5434BCC08458788888AC6C44B0A0787460AF
:20016000849C74707C7850D0743CA4AC5C8498805050A8AC2868A0987C544874BC902C901F
:20018000987464B09C60AC4C84C07C7840C4588088846860CC886C7858B09868A4683CA03B
:2001A0009C54A45850B8703CB450607C88688C887C8C8468C09874489CA478549CAC748863
:2001C0006CB8544CC88478CC48749C94A0606C7898686498307C983C5C804C70B8484CACEF
:2001E000907480B88054AC586880A06CC0906C788C8C904898B46894C474647494AC845067
:200200007C58648C8C3430CC9848609C805068847C84A09458985084A0408C98905C8468F2
:200220008C8860B888749068AC5098982CD08C5490686898787C8888A4685C7CA06C7864CE
:20024000B82C78D868785884B84884B46850D4705C68BC8C48D85C586474B098486CA09492
:2002600030A87C6868686870C0483C80A84088B0503CBC847C4490749C64A4A86C645CBC72
:20028000C03C706CCC9C7C803CA4AC88688C6C809C84506CA0A0805C80B864309CA478A40E
:2002A0004C70B034BC70248CB0904888A45C44BC6078CC50508CA0A8248CA454C4706480DA
:2002C00048A8C0508880B8788444B8745CBCB05470A07850BC5074C88858648894B434640A
:2002E000C8746C7C9C4C5CC87C6C68A860547C6C8474888094A4444C949068A04C7CD46446
:20030000487C7094B470886468C444589C8CC08C607460A8648CCC389CC06480505C90A8D5
:200320009C3470BC8038987C3CB4B4A84C48AC689498787C88A8745C48709C80BC606CB4D1
:20034000A4543C98D080789888445C80DC4050B8747C842864B46C98B46C6888AC70687CDD
:200360007CB088648C84389CA46CA88074A05C6070989074BC9054A068409064B898508071
:20038000885840A09850A4C04430BCA05078B0A86080984C7C6C64D45CA09C40708C9068B1
:2003A0006CCC7870C07854A8646888A48C50908038A0A4946890705C7470588098A0889C19
:2003C0006C506880886890B460687CA0647CB468888074B0248CD84884CC6460688C746489
:2003E000A44460DCA430687084847CB44480BC5080407CA49C6C985C888038D08844B47049
:200400007C80688898788088B43C70984470B0985C70A4348CB484405CA4A060649C546C7C
:20042000D87C3C848C6098D02038C4D08088447C9C58D46854B45CAC7C40B0587CB4683CC8
:200440009CA0704C90A480A0803890986C949C807064789058A04864C094683074C88484A4
:20046000648498A08C345CCC807074789450906470788CA8506CC86034D08C4890BC747CAC
:200480007C485CC86C58AC98548C74748C78BCB4704C84B87870C45C68849464646CAC4888
:2004A0006CB080686C8C6860B45C80BC78548878987C3C9C5490D03844ACB85888889C5488
:2004C000A07C58BC5CA4B440B03C70884CA8746C9070988C60A87C44ACB4685884A8705840
:2004E000C4A4445C5CA0A8844854C0B85054A4985468849C6090688CA8684440BCB8746834
:2005000030B8B458A86884B4487CA86C808C5CD8884C8C689098647080B0744CD88420B89F
:200520006888B0286CB0986C40D04C64BC5C7CB0505C7C88A86C5494888C2C7CD0845C6057
:200540009C90887858A4B86C787C80989850985C909440D8746CA838C89830A894846C743B
:2005600088703CC088648868904C54BC6488B43C80B05C709C847084B84870806C7C9074F7
:20058000A07474847C8C606884A0B84840BC98705C7888A0A86058946074AC9098C4346C5B
:2005A000D4484C88CCA074845C54E43058D898646C68AC3C7C8894AC54409CAC5C4088985F
:2005C0008CB0544C7884587C74A0B47C4C78903C4CC47894AC4080A87828B8E058707C648B
:2005E000D8586094B08CD03C487C807C68C4B050A87C746448A8A48478983C888484786CCF
:20060000746478CC40685880D0885CB87070444CA870B4A47870584C74609894786CD05062
:2006200048A4A06CA484807C80448884B06484E064304C9494A4A08070A48C80A41888E442
:200640003C80DC3C4080A05C8C8C4CB89034589088A49C44ACA8303080A0C46444ACB8444E
:200660004C80709C808CB04C6C5870B8A0984064AC6074983484C8A084388C8860C45074E2
:20068000CC807CA430A08858CC9868986464649CB84474D0807C4874A848B8787CB0504836
:2006A0004CA8A860A88C488884588C88808458B0703C8CB47C548C6460C87440A08824BCAE
:2006C000D4882490B078547890CC5850B488846C58AC98A85438B4A45C80A8748CA45C44F6
:2006E000E48C1880E480584C64C8806488609C98804464D88020D094249C9C6488983C841A
:20070000885C6CA4687868AC5C84AC8884706C6C9884A4646C8C6CA0905898AC6438A8B4C5
:20072000788084A4B85C44ACBC5C60987C648C8C5488A07068A4606C8494847C80A05864D5
:20074000949C4C688C806474686C848C8874788888847898747C8854A8A88C503898D450E9
:2007600054C06074B46470A48C64B49C4C88806088CC604080AC60505CA4B8784878BC8471
:200780005C849494804888A488647C9894547C8C48B47C40B8A0847C708C5894A0586CA46D
:2007A0005C78BC6C687880A43C789C6C906C6C988C8C5C809C54648478C08844788888889D
:2007C0007C945C9C885CB09440A09C5494A0546888B494649058948894903868C498606C05
:2007E000A470589C6C7C9C7064C0804C7C9494906864988C64607C8CA8703488B04450B055
:20080000B44478B854847434A0A07C648860909C7038BC944CB06074C058A8BC644C9CB0BC
:200820008460688C8890A88858A080546CB89470A46860BC7C406CC47434A08C6450709CFC
:200840008C887840708CA4784C84B880703C745C8CB06C68A07050C48C507C889880849CE4
:20086000487098C0885078C4684884A090B4707C9CA06C5488909C8C78689C4C3890A06C78
:20088000B068647C94607074C4A84454B46C64948C60A86844986C60787CA89848C88C44B4
:2008A0006C906C847C888CA060407098809C507CCC78308CDC807C7874E48C1468B8A48CF4
:2008C0009044B864445C9CCC5C50B4B0785C5494AC70944C64C87838889870807480509098
:2008E000884C8CA49C9C508498405C9C7080A490546C9C5444ACA07CA05C5888C0944C803C
:20090000B8907864489CB064809C8868686C80A0707CB48468A05458B8945878B0885098A7
:200920007460888C8C6084A45860A88858A8C43C44A488349C9C7C7C7498703C8C8078B40F
:200940009854547CAC807484589CB4506C74A09070807C88687C988478786C98C85C4C68EF
:2009600098A0686890A4A864409CAC646CA4848478885C8CA06068AC8438889858687CA077
:200980009C5470B03850CC84548CC03864C04C70A86C789480808C806C6494B080886C986B
:2009A0008444A8B844749C68506C8C946084A07C64849C806888809C8C747C705C90AC7073
:2009C000608098746C8C8C6480B87860C0703CB8BC5C5070907084705C907C987060BC6C4B
:2009E00040949C6C809088647CAC705C6078A874587C707CB88078788C7080B0745CA87C2F
:200A000064BC6844B09C686468A08C9474709098806864AC94588C947070A08044749870FA
:200A20006CA4885C64CC8C34B48C349CBC4044A0A49C505C7894707C905078A47488A464FE
:200A400080844C84AC885048A8A4687080809094886480B06468B47C7878748894A04C64C6
:200A600084A08064987878709494749890506CA4944468AC844C94885CA08C6858A0A8608A
:200A800074986C6C9C6C74887C7C5C5C84847C68947464A07C78AC905C70A08494784CACA2
:200AA000AC4C649C98A068309CD0585CB87860B8585CB8A8485CAC5C74AC54688C84786C76
:200AC0008880849C7C4C98A84478A86C6C80709C7884704C84A074746488B0647098987842
:200AE00070588CB06864848C9484787C7CA47C588894986064B08474749C5C74906C9094F6
:200B000068846C9894884074A88C945C60948C74885C5CBC94605068B8986480887C886035
:200B20007480786C70B0A4446490946880A05C70A8A0705C80BC98606078B06C4888AC8CB5
:200B400058988470888478907C94A84874C4583498B85C48AC5C5CAC5C40B4B0806C549005
:200B600090789C8888707C88588C8464947C8CAC605094A8707080C09C64646494A0787C3D
:200B800068A48444705098B85C807478C04C48B09C44B4B054607C60748C848088748878D1
:200BA000486CB8B08CA4805078AC846C90AC6C8468747C7470908C9C94584C94887480801D
:200BC000A0846C707C686C98BC6874845848A0A45C84A884A06060885098C86C5490844C69
:200BE0006C90848C6CA8646C80684CB4C87050949468705CA0B4688C8860788C6C70B080F9
:200C000088886C707C7098908C847C587C8C846070ACAC7460804C809C9C5C78C86C388024
:200C20008C5470B8905054A46C6494A0845C949C5064788C8094B87C5858946C60909C6420
:200C4000849C7064B86860ACA47478788C7C70786CBC845C707480805C80C09C7C6050A488
:200C6000807494908478904864B8584CA49080607878847084C48434B498347C9C8C7C6CC4
:200C80008C5C887C3874BC98644C74C49850A070949C749C606C9C4478B47460809880689C
:200CA0007C80A09C707C7884A470709C84884C788C60A06854ACA060788068A0A05C6C6C5C
:200CC000908078647488785C788874707884847C90787068BC9C406CB0A85058ACA8407888
:200CE000946C84B8705890C0804898A07C785490A46484887498904C64A8A064805C9C90B4
:200D00006C807880847C7060846458A8945C707474A050989C6068C47C3484AC58988C4C97
:200D200090B0806C6080D47C287CD4884074AC88A06C50908C60704C9CA44C80B4984058EB
:200D4000B0947C90746C98B0604C94B84C8484606C7CA898487CB0844C78A48C5C7CA45887
:200D600070A454489C8050848C849C5064ACA478846474C0804088A8B44C54B0845C608CCF
:200D80009C7C84986C9CA45448AC9490745870A05478B46088A04C5898806890A06C94844B
:200DA00060788468A49C407CA45460AC6C88A064A87C788054B488687C7C9480845848A88B
:200DC000A080845860B47C4078B49C54788860707C84909C6C8C5C74A87070ACB46858AC13
:200DE000846C9864789C846890586880A484748884686C6C80A8886C90A4847048608C983F
:200E00008464748C8C70608CB4985860B88044789C94987C70688C54508890809888787816
:200E2000787090848CAC8064587CA86C70B0545C9C9450549CA878987C6C98805C7C8C90C6
:200E400098887C98644890B46C58A088747C6C7494989C84746870687084A8946C906850CE
:200E600074749C94649088788070609C6088C888783440C8A44460ACA868645C8078B0849E
:200E800088B4744C54889C8C94788C9C6868846098847098A48C44688898B47868985C6C56
:200EA000708474949C8864608C4C70AC68689CA86850846C787C8088A04C64A058907C68E6
:200EC000A8A4844878A8887868A8C480585454B49C648CA87C7C64586CB88844ACA4486002
:200EE000A47894985854A0846C6C5474B47C889C687CA05470BC887860A09050849C34743A
:200F0000BC885C4884AC5864A4A07C74786C90A04850B8C0643874AC985058A0B47C447C19
:200F2000B4947888849894647880A4905464AC9850707C787C849078789C6878B06C4C987D
:200F40007C706080945444A0947874647880946C609CC4785C949894684CB0945C90644839
:200F6000B0C43C5CC48C585C78A0B85C44A09480685CAC8454746870A08880947078909065
:200F8000806CA49488787494904C5CC07054A0785484A45C5CB49C446C9C787C68749870A9
:200FA000945C64A46064688898A898686C80907C5C98A86C708090886070AC9470A05C546D
:200FC000B480788880A4984C608890686C909C58709C744464C47844AC8874885C7074A449
:200FE0007C58809C884C48C0A05094A06070787C9498988C68849C604070B8708490548441
:20100000A868709CA47868988460747C90BC4C5CA46868907080547CBC9C64647C80649CF0
:201020008078A8805C4C889C588490608C7080747CC06C44C0B0405CACA46C8484988C64C4
:201040008C6C54989C78787C847480AC706488908054588C9468748C6C845C60B4805C7C28
:2010600074889C7854B088607890A4885460A098887474909890606CAC7C90788084548058
:201080006C90A4904C70A07C7468947478A884646C7C887480907C6078947854947868BC84
:2010A000784C988C5C98AC5464A4887C545C9CAC705898B86C585C88B47C78947870849058
:2010C0006474B084507C9C745C8C9C7C8890707C90845488A8807C7C70807C907068947834
:2010E0007464748C707494607C98985848A09C70707C907858749C84708088A09080585890
:20110000C4B45C48A0C86850887CA8905C849064648074A4A84460D46828B88854A88C749B
:201120006C50B8A4408078949C7C7C4478BC7064B0887068788070949C50A48458646CA8FB
:201140008C846C6C9C94445490948074748CAC7040949C908C707488845C8C8C78B094609F
:2011600058B0A03898B07C80888C8454A06C58BCA06C54749868747868AC8C6868708474A7
:2011800068709CB0645860849490607CAC70689C6C589C847C8484888468849878749C806B
:2011A0008C7C547098A8944890B4586C60747890946874A89054789C709090807080786C6F
:2011C00074809C846064986C5888807CA870508CA8647094709CA0606C74A0586098888C63
:2011E000807080888C906088A88C74905870A0888878588C7C54888C8054A0A468946C5033
:20120000ACAC845870908C886464887078907884747480888088806C7498887870B08454DA
:201220004C8CB050588C7C80948480948864748C8068A89468606CA09870649470508CA0FA
:20124000807490788C8474807478A49050709C90784C949C58846480B88C4C789C7C8070BE
:20126000708068808C9C4854BC78509C786090A47C78A4647CB064607878987C8C845898B6
:201280008C68886484AC606490988C746478888C60647C9874608090886C808C947C487CD2
:2012A000B4908070708070846074B484806C54B4A84864AC8860A0847490848488746C880E
:2012C00068708488805C88B4745C948058908848A0B07C845864908068A488588C985C549A
:2012E000A09C787084A4745080A89880605CAC9C4C4C9CB4605C94B05C68906864989080EA
:2013000084848C885C80AC7C7474889064809064AC7868907C8488706470B48C60888C60D9
:201320007C7468B090584C80748088648494787C6878A8A854589C906C7C909C8078805C15
:2013400090B474487CB07C4CAC9C748070888C88807C747088886478849C605C8480809095
:2013600080588CAC70646C98846C9C9464606C907C6478887C889C6080907C84907C548CC9
:20138000B068547CA8B86048989860648898809080648C9478747094A0606CAC7C60786871
:2013A00074AC9454808474808088946470907854949874708C9868687468948C7C886C8C65
:2013C000904C5CAC747888907C747C74B08468AC6070A490605888B48860709090585CA435
:2013E0009C7C8488A46048849084AC804C6890A064787C64AC84507CA084746C7CA87C5821
:2014000064847C8088748C907C8078647C847C98948854649098A458749C748468609490F8
:201420008C90845C84746C848C7C848C6084906068809C9C70788474806880B07464747404
:2014400090885C9C946484B454489C886C988088A46470806074947C9478884C58B0848CAC
:201460007864B49C586474848890A878688C60688498A04C60B85C547C849080A4886C74AC
:201480008880647CAC78709C78708460707898AC804888A06C6C94AC84787C54808C707C70
:2014A000688898805C6C9070889C908C706870A87070808CA47C687C9460649C7870908848
:2014C00078807064A88C808C646890785C88A0746C848C6C7C8C7C80987C6C908C784C7C6C
:2014E000A0A47460908C686C7898986874845C98A46080907C7C547CAC6068B46C5CB090DC
:2015000070708C84806C6C988C788470707484905C948C4C947C7CBC78548490907468742B
:20152000A47C547894A04C509CA8805080A0808C74708C94845094AC6070789084607C84DB
:2015400064B0904878B4985C949C707888845C68AC8058908C6868808C6880A05C709C9497
:201560006C6890907C787C6C6C94805478988460889884904C78B894746C9880648084A08F
:201580008C84705098745488B8985864907C6CB06C6C9488947464888084984C7CB8685C97
:2015A0006088B868807C549C74787858AC8C5898A4605478A47C74807098A86C4864A0B453
:2015C000844C70A4906C809898887488746474747CA0847088588CA05080A494807C90780F
:2015E0007088747CA0887464707C70AC684CA49C8064647C8C74A4907494586C8464948443
:201600006CAC8C505884889894787C84847C84848094945478A85C58987078A878787C84DE
:20162000807878989C4C74BC80488C884C94C0684070AC8C5484888C7070946088B05474FE
:201640009C8C7C507C847480948C7488805C94A06084887890605CA4A0707C8478688088AA
:20166000688CA06484A460549C90807C5CA48C4870B074549C9890707C90488CBC645CAC76
:201680009C445CA0907C6C887C7C88545898A8846C80B06C5C80948080906880A06C5074BE
:2016A000A07C8C94806C5C78A894687888908C78607C7890946C7C885460888C806490B81A
:2016C00088505C8C88649C9490844C74A0887878988C705474A480788C848894805C7C883E
:2016E0007C7C909C74786868887C74AC70548C707C7C748078A4984880A080786CA0A46C0A
:201700005C70789478748488A0745480A0906080C098505880A498746C6088A84458A49005
:201720005C74B888486C8CA08058A0907094845478946880987C6870807484887CAC8C68D9
:201740008870848C8C7C808C74485498947470AC8050887060A4A86470A894604CB0B85CAD
:20176000408CAC746C787870B498408CB4686488A47C6084B078509C744878A888689464B5
:201780006898687C948CA0685C9C987C5870A8A064547C987C789080808C74648888746C7D
:2017A00094948470609484689C6864B0785484989868609094746C8488807C6864A8A0604D
:2017C000748C747C9CA47870787864809C847474747CA07464889C8464586C98BC8850842D
:2017E000A05858A07464A074749060909C5890B05464B088688C7878988470885C90904C35
:2018000078AC8C788878587890749098807C84907C5C648C8C908C5C8484789C84788C84A0
:20182000884C589874A49064A89048647CA0906070A08C507C9874709088607C907058A414
:20184000A8648480808C788C6C68B09C707084786088A85880B86C7C64789C648CA870786C
:2018600080548094707C809860487C74A4905C9484808C6078948478908C6C7878748C88C8
:20188000608898748078807C749C8C84988474608C985080B09044508C7470A0A07C606C90
:2018A000987870B8704CB8A450747088885C88A47C706C7C7890A86C78A8904C807C7CA404
:2018C000786894784C80A464788C847C74947C58847C849C907C6090884C84B484747C8448
:2018E0007058A0A0648CA4845058A488749C787C886C78787C907C7894906058A0A0586830
:20190000A86C7484786C64A8946C8C90885470BC7048B0A0746C748C4C70B8B05C649C80BF
:2019200060A08C5C90A8745468A4985C70A4945054746C80A48C5C6C9494806C98786CA0EB
:201940009C7474807090907068809C80587488849C8870787C9C88607C9C7884946C506CCB
:201960009490746C9C8C5868A8806094AC84647888807C70808C9494585884988C78808C4F
:201980007078846C7CA0788C846C806C7C8474947C6C88808C7860607CA48C84946C5878B7
:2019A000849CA8747474687888707C94A07C5478888470889C74888C689C80608894909CDF
:2019C000885464887C786C78989858549C8868849C7454988C5484748890948868688864B7
:2019E00064989894806888805C98AC806C847C7C90745484A4A06860647C987C70988474EB
:201A0000746C749488647CA48858809478646884A874708C5C88B0745488B0745C886C8422
:201A2000888C9C747C8C64649484807C88906C7488705C90AC685498745CA08C747C7884DA
:201A40008068A4845890A8904C64B87C4C848C848C98785CA484747870A88460948474807E
:201A60006888746080845C808C6868A4A44C6CA86074A4808878708894686C88908C8470CE
:201A8000709C986C90907078848C9488747C70848C6C5880988C5C7490846870A89050588E
:201AA0008C9C8C947C648088705C909C6C5088A07064A08C6884746C8C90A4785C84947C26
:201AC00070847C7088887864809C647C8C74808074886494AC7C5C74748C7C608CA8787852
:201AE000906C6888847890886488B0807080789894747064688C885070AC70688C7848647E
:201B000094A47C74A89C64707C7098AC6C74806C7070888474809C7C5C6C9CAC84889C5881
:201B20007CA478605C8898A07858907C6068749C947084A48C60609CA07C807060907858FD
:201B4000748C80807C74785C8890789CA470708C64789C6C84A0747C7C5C90746494847CB9
:201B600090907070AC8464A07C6C986C6088888C806C84887070647484A094587C987458A9
:201B800074A8845C848C7C707084887C7C5C8CAC7458847CA09C786C747C6478A880748869
:201BA00080785C68A484609C88747894906474986C7C84887C6888807C9C788C8458706095
:201BC000A4AC6C64888C7C646894A4707C7878A8845888A08078847C848064809070687809
:201BE000808060707C8C888C74749488546CAC7874A89C5C74987070A494707084887888ED
:201C0000A0785494A8545C948C746C7898646C94546894806890887480787098A4845C8030
:201C20008894A068708880807C7C8478607CA07C688080708498707C8C7C888C74708480B8
:201C400070707C8C7C686C907474A080548CA8785C8C908C8084805C70A0906C7C706C8CE0
:201C60009C6470988484847488948474647C9080707C946874845C80A08C60748868849494
:201C80008488908078707C985C90B8544C848078889C844C80B0885074948C708088708470
:201CA000786484846C809C7460847C749C8C789880708480847C8080708C9C787C74608460
:201CC000789C986C6C68807C848C8088845C787C8C906078AC6850AC94587084A880608C38
:201CE0007078947C7C708C98749084707C808C78648C80749060748C8C98646C9474808014
:201D00007C848090887C6464989078706070989C70607088A0886488948C78847C789460F3
:201D20007C9474887084885494A86864887C688CA0707894887064809C7C6488846C7C94CB
:201D4000887080807494886C7C948074887C849C7C6888747C90787870708888707C7C70C3
:201D600074909C6C5CA0905864A4A07878707C9C7C74848884787C90806494887884749C43
:201D800070649C807088785888AC6454888C6C7878808470707C9C90747C889484687C8CA3
:201DA0008C84707C9888707C848884708090747C8C7C88A86C509CA45460987C70907C584B
:201DC000789084747884908074907C6C8C90847C80806C747C74909C64749C805084B07CFF
:201DE0007C8C8494745C70849C8C5C689C78586C749878809C545C90848C90749094707C37
:201E0000786864A4AC706C7C7C948074807C8CA48C5C6484847884847C80886C5090A06CF6
:201E2000609C94608474647C8C8C84A08C50689C7880888488989058589CA0706888A8789E
:201E400058848084808494787C6C588C8C7C88A4886864786C8C9864849070747C70747CFE
:201E60008CA0886480947C808C5C7CA88464647C8C748CA078606C7474806C74A0A4785C96
:201E80007C8C8874748488905C6C94787C6C80A48064807C748C987880AC705498A0707C4A
:201EA0008C9074707C70788C80847C88785C9CA858689C8C8074647C84887060A0A0584C96
:201EC00084907078A494787470889C6C74A8906C70746C94846090907084645C949C6C8012
:201EE0009C88607C88889C70709890706478A0706484949084787C807C80809488788460DA
:201F000070AC705098905C706C70908C687CA890746C6C94907C8C987C546C9C885C789801
:201F2000906C6488986C749C88748C786CA0887880749C885464848074946C84A4746C78D1
:201F40008C8C6C7C8C947078887880906C60A8945C6478A0946890A8645484987888946489
:201F60007C88706C7098947068887C687C908068709C887C7074948C888C849484606C9C81
:201F80008C689CAC78586C709484688084907060847090986880946C6868647C9C90687CB1
:201FA0008480646C988C6C949878787474949484948480886C7C947C70988C707C78748801
:201FC000747CA080706468748490746C9078748068806864A498787870948C7C708CA06C5D
:201FE00068907C708C8C8C8870908C707488906068A48864706C848C886C6C8C8480685C51
:202000009C9C686C888C807480807C908068747C8C90848474849880807C6CA49870846498
:20202000689C90806C64847C707C807880888860848C748C8C70788C905C5C809078689C04
:20204000946C80A484508498948C7C7C60849C8860649C8C586884747C7C8890888C806C98
:2020600078988C6C8CA0745C80846C848C80787C846C7C8C9080889C745C8C948084807454
:202080006C78746C7080847468A4A46464988C6C7C9C8870707C80848C6C6CA090585478D4
:2020A000AC74749C9074708478849088947C68785C80A88C746C90A05C58A09C648C9864F8
:2020C00074886C848074808490785C6480806C90A490746078888C90747C98887470807848
:2020E0007C948C8480706C6884807C989C7C6C5C648C8C7C84987C6C6C687C988494A074F4
:202100005C8484788C746C90A8705480987C70849C8870705C78947898907C9C7C548080FF
:202120006890A094706474687C948090988060607090988070848870845C64A484809878CB
:202140008074747C94986880A48C5C6878748C948878787474786C7C8C84907858809078CF
:20216000907C94A45C707C64888068949C746488886C88A0747C9078687C9C887890846067
:2021800068748478749C88646C8C9478708888789890707C74688C946C688C806C84806CA3
:2021A00080A4946C647490846890A88478745878986C7890788484747C80887C8894806033
:2021C0006890888090708490787C74688C90848488687898606090A87858809868747C744B
:2021E000889474708C7074948C7878908C6470706094A8887858788880886C7C908C80601F
:2022000078948C80888060809C7C5C8C84709494807C6080A46C6C988474787C68749480D6
:202220006C80787094945864A4987C8488807C6C989480706888785C888478989C686488CE
:20224000847C88887874748884647CA468648C846074A08468949C74788C8074848884789E
:2022600088846C7C806C7C848C7474848C7460849C7C88846878888C6C70948C70707490AA
:202280008460989C748C74748C847068849084706C9098647490707498786C78846C5C9896
:2022A000987C846478807C947C708C887888848C807488846C749C8458889C6880A07C7C0E
:2022C000787894787484847C70989460708468748C886C688C706C948874849C8064748C5A
:2022E000887C807C847C7094707098847090A0746C8C887C887C78988C78745C788C786406
:20230000749C746884707494B0906C68707C8088986C7CB464509C7C5C7C90907464989CC9
:202320007078847490B070507C8C707088947C6884886C688CA08C8C80648CA06C5880A0BD
:20234000A07478845C6C888498907C70707880989088846C648C8460788C8C74808C607CBD
:20236000846488888084647CA87C548898808484707C9080687498A48054889C5C70A09059
:20238000687CA46068887080A8846C6C7C705488A87460908C68688C9084887C7870787CC1
:2023A000787488A0906874888078807C9888748C886C7C7474A89C64687C886858849C882D
:2023C0007088707094744C8CB498644C748864709CA884707880787C6C84A89060708C8849
:2023E00064909474707C8C6854849878888C74889874586C8CA094888080706084847C900D
:202400007C74807C6C647094AC806498845084A080888C706070807C6884A0806888885C2C
:202420007088887890A8706490845C74987C58788C707898806C90A8906C6084987C7C88A8
:20244000809C98745C6498885C94A06868787C808C80888468887C6888887078706C8074EC
:20246000807078A498647094847078888C747CA08860848474808C7C6C78987864949C7854
:2024800080806C74707C78849C9078647C7C7C8C88748884847C748C847C80708C88647C80
:2024A000887874888874808C60649C8C8078687C8070747C748C9C9474748C7C6C80888C50
:2024C0008470847C8C80648890747880746C7C90848C94707C9880708C90848878647C9000
:2024E0006C747C68908C7C8C747888707488786890A4745880A0885C688C8878847C848C2C
:2025000080988C707C7070908C846888A474646870A48C586CA494707C84848878789490AB
:20252000748088847C6C849888685C889C7C70949874647C807064889870687C88908868EB
:20254000646890A464609C9084947468808C70749480648894847C708C98786874848C9883
:202560007C687C8474748478748890807C88707C98706C8C989070747C8C84686C887074BF
:202580008C9090707C8C9C7C4C8CA8785C6C7CA0AC60548C986C647C80848894807880902B
:2025A0007874987874848890746474888070708C9888747884788094806C7C887880946C4B
:2025C0006CAC98585C74847C749498787C8470848C686498A45870AC7C547890988078782F
:2025E000607C8874809C9C786C84848478748C8C788C74608C80649488707C807C6C747C2F
:202600008C8C888C7C706C84A0847C80787888745C90988C786488887078707C98847C84BA
:202620007894805084B084508CB44C4C9C8C7890987874906C688C8C947C68887C688498AE
:2026400070749890705C787C7C9C848490807C8080847C787C807C746C7088806884907CC2
:202660007858609C9C786C809884645C84887494987C747868849C987878888478787C888E
:20268000809094706C90746C88A094687C886058889C6870A080646864848C6C8090808092
:2026A0007C6878948480A0986454707C7C8480809890785C688CA4A4647CA05C587C888C4E
:2026C0007C8884786C6068849C8C7490987470849C807CAC8050809C5C5884787894987022
:2026E0006074907474849098786C6C708C94787CA088585C7C7C747CA49C6878847C848422
:20270000708CA880645478987C80809888547C946C80A080809474748894805870A49460C9
:20272000707C6074908C808080887878787088A0905C58909864789C8484806C68789078F5
:20274000809C8C7C6C8490707C88707880686C889C848490887C747480847084906C74789D
:2027600084946C708C887C847C5C849C6480A0788C7C648C686490947C6C7C7478948C7C89
:202780009C9C78807C6074989C80687074806C74A07C6C8C846C70848C7C80886C74989049
:2027A0006460888078847090987C84787C9C907C7088846078908C848C847074746868747D
:2027C0008C8C787498806C8878808C74707C9090748098807878809070809C705890A474DD
:2027E0005C788878688C906C888C6880847C807888887074988C70787C707498845CA8940D
:202800005C889C98685880908C8C6C687898987074886C6C70849074949C706C88808080EC
:20282000887C747474707C84746C84847C70809CA06C60909C947C58849878706894A46CC8
:202840005C747C747884989C7084907078846C7CA0705C78808C8070949064688894847CC4
:20286000848490987C6084806C887C74787C7C7484846488946874A0987858849C8070689C
:20288000709494847474848C8C5C78946C74949478707080A8905C7098806C707C8C989820
:2028A00074647C84706C7C8C847080885464A8A080846C70848C706C9C8C70808888807478
:2028C0006C8890708490747080849088748098805C6C686890947874A4845468889498A004
:2028E000848478686C749498787C907C5C5C78A08C70787074847C80988484A0A06C687C0C
:20290000646C9888889C945C548898706C9490806C687C8478788894845C506888808CA80B
:20292000947C70746870A48880A4846C7080888C90787C78787C786888A06864A88C5878BF
:202940007C7088988870786C7080808090A0907C8084648490708C9C784C648C7484AC9463
:202960008068587C7C8CA484789898584C8098748C8C5C74806C74908C7C888C6C789C7CA3
:202980005474A4986C8084587488848484A094707C80647CA8A080889058507C7C6890A843
:2029A0007864606478908888907880786878848C989484708070688C84788C98807C746873
:2029C0008C8C78909084806C54707884A4846C88844C608C90A0786C9C7054787478B4B003
:2029E00058609C705498A47078A888606C6C8494889084607088747490847088988C686C3B
:202A00007C7C84808488806C68788484949080808468648C8C88A890788864689078848CAA
:202A20006C6C80705488A47C70846C6C908C6C889C7C70808C707084847C6874887C789412
:202A40008C6870949C7C808C808094785484A46C5478949078748894747C88646C94907C86
:202A6000909058609C9874686C84747080788C9894746888847C7C8888787490787C8C6C92
:202A8000788078887C7C887C64848C787880806C7C8C6874808C9C887864789C7C80947C62
:202AA000987460808C8080948C7C7C84807C8C9078708874608084788878686C808C747462
:202AC000787C8880788C8890A4685890948080748C6C60908C7C7C88888C8C6C808C888CC2
:202AE000887874889084606C8C78707C8888708098707094808498806070787C8C7484A0FA
:202B00007058687478809490788090847C789CA4787C907C647884687490946C6894805C11
:202B20006C8898887470748478787C949C78807C7880687C9488989C7C708C887894987055
:202B4000806C5C9880649090787470787C7C80707C88786C80846C747C98846C7C808C7C01
:202B6000888C7480988C8890806878A07C5C788C80707C8C88909C7C6880806080A48C6035
:202B80005C848C7C7C888068747C74808494A08474908068808C707C9884606C987C5C8481
:202BA000847C8C887864808C7C888C9068688C706C8480909480785C78846484A4A4886C25
:202BC000707470888C84908468687C84808894947470706470787C8CACA46C7068707C7C51
:202BE000987870948068607484789CA8686C7C70748090A094807884745C7884A0B08068CD
:202C00006C546884849098886C5C707C7088988C8C7C646C8C80889C7C888C647C78689C10
:202C2000987084A0846480747084A08064948860548C905C788470706064848C9C987C78F4
:202C4000807C6C909C7C78907C6C70788C8488846C7C888078748094A0787C84788C807C68
:202C60007C80887468707888886C84A0885C5C7088948078808464689474648880909464DC
:202C800060787C98A08C7C8884606C908890A08C74748078788C80789C945C5C6C8C8C703C
:202CA0007088887C78847C6C8C90948C6C607C90786880A0987864687C8880809CA47C7410
:202CC00064709C806C94946C6060789074788088906C7888848480808C84908C7C78748C24
:202CE0008C847C786C747C7C8080A0A074748C847074908C6078847888785C648090686054
:202D00008C8C747488908070807C848C7C748098846884A480546CA09C888080909C70687B
:202D200084787480749498706C8C846070887878847478849484749084586CA08060708CFB
:202D40009888707C947C78846C78A48C608CA0605484A480787C74848C908874749884606B
:202D6000889468748C88685C789478607C9088809088909070608CA47C687894905C78906F
:202D80006070887C9088687C9C8C70807C8C886C74808480747C7C748C74709C906484A84B
:202DA0008474788094785C747884987054788C7C68587C8C809CA074709C946C7490847C67
:202DC0009C7C647C8CA0806C988C6868908468847C9494606C786C6C84888498805C6C8C33
:202DE0007C6CA09C7878807C7478789C907878707C8478788C888C8874646080A0887498CF
:202E00008C6070887C5874A89070849478647C948878947860807864709C94606888846C32
:202E20007894948CA47C5C8094887480909074708868606C887C84947878808080907C748E
:202E40007C70808C746C90986C70947C5C708C90808CA0947C787C74909C786478786C789E
:202E60008C806C78806C7C907074A8A86C648C986C6094807C988C7060748470648890749A
:202E800074907C608CA4887878888C6C68808C9098907874685C70909498786C9084546C6A
:202EA0009C88908C748068507C8888A87C58707C707C8C8C84949C8C6C60708CA890748CEE
:202EC0009470545C8C7C70989C7870807C749088949C847068707C90808090806C605C687A
:202EE000848880889888605874989C78889C7C74607494747C908C948C6C787C80A090848A
:202F0000946C607874888C7C8C84746C6C6468848C989078707C787C74809C907C70748815
:202F20008C8080948868607C8870749894647C9C746C7C7C70809C88646C848488788C9CA5
:202F40007C7C7070948884746C807C6C747C7C788090906C7C94687890949074707C8884B1
:202F60007074888C84787478787098A48870747474987C5884A4885C6070708088848884A9
:202F8000806C6C8480A09C8C806C6C94885C647C94947474746C8CA08C8884807874688055
:202FA00094848C906C7090785C68988C8488808480706C748C986C7484685C5C88A8887061
:202FC0007C907C68708C949CA0806C6880786C8C88848C88946C5C8C9474787C88907C74E5
:202FE00080706898846C84705C749C90808C908C7878747C84948078907C74747874808801
:20300000787870709098847470848C907860788C6C6C887870787C88787090907C888C8CEC
:203020007C90905C78A4886C7084987060787C7888947C7C807888B09460647C9C78607CB8
:2030400088706068708C8C80706078908C8890A07460909870689088786C6884846C7888E0
:2030600090A4805C98A47C649094646C887C748074748884747484907C6C6C88A0787C9444
:203080008478646C808C886874947C789084787C70809C8C64649094787C88747C8C707088
:2030A00084847C7C8088847C887864848C808074808C84806C789C9C687498806884908004
:2030C0008C747078747C7874809070689090706C8078789080708880787484806888908060
:2030E0007C806C709C9C88787C7C686C808888908C6C7874708478888478808484788890E8
:20310000888880748870609888547CA080806464787888807C8CA88C54789C7C8494846CDB
:20312000788C74688CA08068808064788C807C84988864687C647098887C809080647894DB
:20314000888494746C8894908880748C987C7C6C6088908494806C747470746C8C986064A3
:203160008C747088907C7490946C5C84A07C74A48050808C706090A8806C807C747C849063
:203180009484846878A0886464908C6468908874707090A0847C78586C887884A89068647B
:2031A00074706894A0809088748484747884A8A468607C645C84A490647C80686C7884844F
:2031C00094988470786868707C948C948C70646C74909C9C8C707490705C9CA88C707070F3
:2031E0007468607898949098786880747098A0848480645C6C88987C78807064688474844B
:20320000A090848484706080A890687494886C5C68849C8C888C6868848880809C9C786492
:2032200070605C94A8805C708070707C888494988088887888889CA060608C7C686C7088DE
:203240007C708C8C746C6C748884908C80807878848C7C687884786C70808C9C947888848E
:20326000606C88988C7C7C7C6C7C807078848C8068789084749898788C84746C7090908072
:203280008C8860749060649484887C749880606C84847884847878847478A09C807484885A
:2032A000585498AC8C88887058688C80788C847880847878889090847478806C7890807056
:2032C000808C6C748C8C807C80809C8C788468608080788C84686874807870909084947422
:2032E0006894988888807C746C807C84A0805C6C9088748088847890A47C608098807884B2
:203300005C6474808C807C74686C7C8C888894886C78888C8868708878747C787880889025
:203320007874887C94A46C5C90A098887878746C7C786C84989064647C848C8874808874A5
:203340007C8068888880847868686C7C9C80708884888C848480888C7C6C7C8C78607C8CAD
:2033600074807C788C88886C68909C8C8C886C706C809070687C807C706C849C90607C9C7D
:20338000807C807C80908C8C686488847C8C847084887C8C84747878788474747C888C7851
:2033A0007474646C887C6880948C7080A08864608C9C848C847C848890888490785C787839
:2033C00064808C90947C707470687094A0888874688C74709C8C707C707488787480908421
:2033E00070788C74688888889080887C5C5C78988478908084846C7490A09884746C8088E1
:2034000088808888687C846460707C848888847070787C8C9C8C747C8874708C80848884E4
:203420008480746C789498707C9C7C7C88646C9C9080806C6468707C787C80888C6C608404
:203440008C8C947C9098846C608C8C8C94707078646890948C9078707884888C888C806C38
:2034600078947860808C7078808884687480688CA080708C745C888880887C8C80645878D8
:203480009894A4946C748C787C988088947C5C6C6C749090807C848870606894A478708808
:2034A00084705C6C8C8880808C7068807480A89C80909084685080A478809C7C687C746850
:2034C000889078909870586C989C78808C7C5C5C647898988C8070747C7884887C889888F4
:2034E000706C80948878786888947878807C8C78809C886C58808C787C88A49858587C8018
:203500008088707C987C7880809094846C6C7474889C8C7078909064647C88887C808488AF
:203520008C7484847480787488806C789874608C8C888868707C849884747C847C747488CF
:203540007C788C8874747C888C746C849C90646C849890706C807468747C788C90807C7CAB
:203560007C7C7C949070707C8884788480646C808C7C888C748488809C9C7478746C8C7C57
:20358000748C6C6870648C806C88807C9C7C5884907C84988460688498887C7C78787C8493
:2035A0007470A4A06C709C906480987C60787C648098847470748878749484749094708023
:2035C0009474807474947C7C84788884747C8478807C78847870807C847C68686C78848463
:2035E0008884808C8878786C7C9C8478848070748490908084746078907C889C88707C74C7
:2036000084846C848C7C7C807474747890887464749C94646490808884708C78686C6C8826
:203620009C847C806C748888888C988874906C5C909C94806C78746880807C8C7C7088946E
:203640007C6C788C9074749C8C646878848878688088808874749098908078907468948C7A
:203660006C78A49C705C648C8078707098846078989084787874706C7490807088848084AE
:20368000706884888484808C887C848C8C9488747874848C78908C6C6C88886C5C70948C32
:2036A000747C94846078846C94A0807C80745870A0886080906C607C90949C8C6878887446
:2036C0007C7C8C946C7CA08C60606C9C9474847C8080747C848084907C787C686C8884781E
:2036E0007C847C6C7880889C907C788894706088A88870988C68786C6C807870849C8860E2
:203700006490A47C687C7C7474687488908C748884587C98807C7894AC88547480889C6CCD
:20372000749C88787C68708480807C747C7C788088888898845C648480809C886C7C8878BD
:203740007474808078909C786C8498806488A08068787870888C8C90888068608898787C75
:2037600088907C5C7094685C98987474786C7888847C849C886C68849C84848874787C7091
:2037800070848884887C80847068787C949C8C7870786C7C887880888878647C887C788469
:2037A0009C8464889070747C80949074605C808C78A0A484686878807078907C748078883D
:2037C0008C7C7474809C8464788074748C9C746880786C687C8C8CA4A47470908074889CDD
:2037E0008868849C6C586494946C748074747C707494A47C5C8484807C748C946C6C847449
:2038000074707094986C8CA0847468709C988480707C8C886C6878748C8C786470889094B8
:203820007C849C8C786C6878889884646C6C687C7C7C88848C906868949C8464748C988CAC
:203840007C7C847C7C806468886C80948088808494947C687C7C6C6C908C74706C74787CE4
:203860008474688484809898847C8C907C6C74808484806C7084887474908478808084844C
:20388000848878708080747C7C7C78889474708C887078949480708C947484807880746C50
:2038A0007084948C74648894787C887870807870807C888878786C7098907474788474805C
:2038C00098907C847870808488746C8C8C748084788890907C68888C8078848C706C8C80D4
:2038E0006C7C7C706C7C7C68688CA068608C8C7C848488848878707C989070807C70909C08
:203900007C7C84787C808094807884747C8C747C8070887C647C806C80908C8078788884E3
:20392000747888848C8464788C7C7C7C88986C60888870849880788C806C848C70687890BB
:20394000987C78787484847488A084687070787C8C9484807C7070708898907074786C889B
:2039600088748C887C7C787874887C708080788C8C7C6C648C947C848074707C74748CA077
:20398000907084846C749898847C7884888068788C8488746878807C7480888C84687C8053
:2039A0007484887C787870808078848C90887074807060849C787480949C8C7C708094840B
:2039C000707C8488846C849C8C7070746874807C909C8C7078806C7C889084646C8C807037
:2039E0007C74848C7C64607C909094988C78787884807C8084947C647874706C6478889017
:203A00009488806C6C98A0887870888060789C949C90606478747C7880988C888880807482
:203A200080847C84806C70887C64809C8C74787C746880948C78748480747470808C847CDE
:203A40007878846C607C9894807080808C8C848C7C80907470746C949C84806C78886C7C8E
:203A60008C7C88887C8068649090848C74647884848C7C74848C7C8080708080708498805A
:203A800078806C70888C948C7078806C707C84909074707868688488848C70788078848C82
:203AA0008C8C8C8C80687C90707C88688C846C848488947C7890888074787C78808C9078E6
:203AC0006C78605878A078748C787098A088848C94886470846C688C987868687078708076
:203AE0009090887C8080808080787C887C84847C84746C847C707C78849C847484848C88AA
:203B00006C707870707088A08C746C707C6468949C94947874908C9084687068647C908809
:203B200078848068708C907C6468888C8884848878747C78746C70909888807C78808084C9
:203B4000948C887C748888806C6474786C7084847C808088848080849C84647488A0A07859
:203B6000687460687C6C808C78808C8484888C8C787488806868707C908C787474686C88F9
:203B8000A09C746088A0988C7C8088646884807C6C6C807884907C889084786C90887898F1
:203BA0008C7474687C8870847C5C787864848C809090787C8C8C7C789494706C80686C8C71
:203BC0008C7C6C74887880907C707C808C908480888890906864807870686C988C647C9019
:203BE0007C80847C788C8C8484807478847C847C64748870707C7C909C84707C90848498C1
:203C0000948078787874748488747078707888806C708C88747C8878848C848488807C7CF0
:203C200070687488948C8490947860647C989C8070707888848088786C808874646C8098C8
:203C40008C7C7C70646C98987C8890807C8478707884806C8494847C74888C6C7C8C7C7884
:203C60007C788890909080747868647090987480847C80807C7C7864909C70708084848C60
:203C8000887C786C6C707494A088787C7C88707494846C8094808C807484808C8C848C6C24
:203CA000607884888870747C6C7C7C7884889888747C706C8894848080887C7088887C9034
:203CC0007C707060708C9C90847880886C6880886C6C7884987C7088848090808090787430
:203CE000747C9C9C70808074746C6C88887C8084846C5C748C807C8C906C5C808C888C94FC
:203D000088747C847878948C7C90887078787874747890986C60706C7C8C7C849888747CE3
:203D2000908C6C788C78786C688C8870909C809484606C808C90807C888C7C74807C7C8487
:203D4000706478747090946C70989070808C80808890886C70807880746474888484847CBF
:203D60008074788CA0988480807C707C908C78586068708C8C709094606888808890848C5F
:203D80008C807C888070787068788478787C889498888094887478807C8880747480888033
:203DA00060687C7C98846C888C7C808C90947C687C807C748084705C6488906C5C809C8C6F
:203DC0008C907C7480847C908470788C8C808884807C746C7888807C7C808C80788C8068EB
:203DE00074746084988C98786C7C8494846478988070748498907C6870887C70747C8C80F7
:203E00007484807C847874786C74808C9C8870747C6C788C989C80788C8C6C7094886C60DE
:203E20007088747084847C948464747C787C84909890909C846C706C708484746C847C6CCA
:203E40008C90747480888884746C889C8878807C8060608890788080848C74647C9494945A
:203E600090807C786C78908470687C80647498907068849C9C7C68788094A0847C80746476
:203E80006C887868888C748074789890808C8480786474888C80808C80686878807C78787E
:203EA000848874748894887474809888646C9488708C8488886C6C78808C8480907860742A
:203EC00098986C68989C70648088787878708C88787C7C8C988484846C70787C948C8C88BE
:203EE0007478785C70907C74808C807480888C7C7088845C649080789C908494805858804A
:203F0000A0907074909074707C707C947C80846C6C8088988C849884686884A49074807875
:203F20007470647C78708894908C84787074746C80888094786C8C88788074747458749019
:203F40007C8CA098906C5C848874808480908C6C5C8C9874748084746C80987C7C98808049
:203F6000806C74889494847C7C787474706C84848C906C7090886870808C9C806874788885
:203F80008C748088686C786074849CA87C64807884987078948C806870848088907C848839
:203FA0006C7080687088908C84807C7C849480707C80786C808C7078908C8084846C60746D
:203FC0008CA084687C7C747C808494948868648478808C70789070709C80709894888874C5
:203FE000748078748090846474785C74886C6C889084789094788498909088808078748CE1
:20400000907878846C6880706C909C847888847470808C8870708874607468709C84687C34
:204020007884947C849C88807C7C8888848084907C5C707C746474888484989C7C74888C54
:20404000847C807C70808470809074686C7478647894848C90807C84848088908480808488
:2040600090786080987074748488748C907C888C7474807C747880746C7C7C786870807CC8
:2040800090A08C748C9C887474848074807C707C9094847074807C7C7C6880948878848CEC
:2040A00080807C707878707874687C90888C807470808C7C80807074848C88887480888054
:2040C0007C8088888084808890807C8C84707078887C787860688C7C6C807478886C809430
:2040E00080708894746C888C90947870887C708078789480708C8C748894847874808474BC
:204100006878847C848C887C748078788C807C9098786884887870707C886C646478788427
:2041200088808C88848C908C8C888C8C7C7C7870887C708C80707C6868888874807C748873
:20414000908074787C8C90746C74748488807C84948478848474809894787478807C747477
:204160008C9478646478848074788880848078908C80848C8C786878887C787478947C6487
:20418000707C7480848078889878688488848C88847470887874909C8C807870688090802B
:2041A0008488746C849488786C787C7468849874687088A07C687C7888887C889874708C3B
:2041C0007C80806874948474707888846C648C946C64888C848090947C8484707078889413
:2041E00090847C6468847C7C88807878849894787C8888887870706C848C8C888074606413
:204200008C805C808C8C94808C906C7488808080746C6C747C8090847884806C78908074D2
:2042200098947478747884808C907078806C788084846C7C98908088807894887074707C8A
:20424000847C74848C8484886864747874808C7870888C787080908C847C747888907470AA
:204260009094847874707C989C7C6C70788894847878809C84606474887C809084707C7C52
:20428000848C748080647888808C8C787C808C907864748080748080808C8474687488984A
:2042A0008C807C70788C887C908C848468709498786C7874848C7C6870889084807C706C2E
:2042C00078808078748C846C7C84807C7C8C988C80847C707C949C8C84686C8478706C7806
:2042E00094806874808490787890887C7870787C7C8C8C8C887C787878707C8C8C807074E6
:20430000888C70707C787C7C748088747C8C8C8C8080806C7088909888747C7884906C70C1
:20432000888480808878647890806864708C8884848484888074748494887C9C9C8090844D
:204340007C84706880847C7C7878787C7070807068686C809090887C807C74807C78808809
:20436000887C7C9898687C7C748C847C7C7C8488787C94847088907C6C788484706C808C45
:204380006C587C9498A0706C847C847C7488886C748C8474788C8474787070948C7084984D
:2043A0009894706C78807C78807870747488846C848864688880887C687C888C90847C7C59
:2043C000847C78888C8888746C80787098906C788C908878788084847C848C806C707C84E9
:2043E000786070846C78887C80848880808C806464747C8088947C787C6C74847C8C887445
:204400008894908C848490948074707878746860888C707874747C78888C80908474948898
:204420006874808890787C9084706474989480786868788498886C747C7C74686874909CEC
:20444000846C847C6888906C7C8C8880788494948470747C8484747C807C8484848478707C
:2044600074808C747098946C808080807C7C8084807464788C84807464687C8080747480C0
:20448000909480686C8090888084848C907C80848884808C80707C84848480848C78606010
:2044A0007C807C90787088847C8060609890847C6878949088908C806C6C8080809C9474F8
:2044C00084807078787C7C849880606C909470688484747C84706C8C907C84887478807C38
:2044E000889888908874747C6C7880788498A0886C60708C889090706064808C80888870C8
:204500007470607C947C8094948888806C7C8880808884786874888C80788C947C708080AB
:2045200080909C886C7C7474847C78807C788070687880889498847C908480848084786C87
:204540007478787878847C80907C68747C7C808C9C9C8068789888646880888070788870AF
:20456000709490847C78847C78888488988C6C707C747C78809084706C7070849C98847043
:204580007C90887C788894806C68646880887C887C6C807C74787C90907C74748C9878706F
:2045A0007C8C9C8C6C5C6088988C9494747478787C7080908C80807480887070888C80740B
:2045C0006C6C78949C908C847C7868787C6C88A08C78748478606C7C8C88707C7870847C33
:2045E00078948C78786C8498808CA080707C808884646C88948C74647C78687480888878DF
:2046000074889088888C786C646094A07C788488787C9480748C886C7480889084706C70BE
:204620007484785C7094887088908078647CA07C709094888874809480646084A0805C64D2
:204640008880708084807C6C70949C88848C8C78687C948470748C989484645C8C9464706A
:2046600088787C7C78887C78988C646074907C74787494907070787C9C80749C847478787A
:2046800080707C9C887470686C8C9468689894686484989888888C7C787C708084808C8426
:2046A00078747488907C687484807064748C948C78707C888478787874889C907C6870904E
:2046C0008478807C7C746C78808C9484808468607480908C84908068647490989080747816
:2046E0006C5C7C9084807C8C80606C80849CA07C748078686C8894908C8C88786C7C8878E6
:204700007490907874807C647C9878748074685C6C908898A0847870707C74849C98807CC5
:2047200088747C88747484787C6C607894888098846C747474888478888484847C787074E5
:204740007C849C9C787080848C8078848C847068687CA08870786C686C70889088988C7469
:20476000746C789C88687C8C888C8068889C8C786C6068888070848C8480746C7C8488847D
:204780007C847C8898847C80808C94706484848094786C8C90887068747C90A09474606C19
:2047A000746C808884847C7060748C7C7C9498786C74888484A0A48468647870587C988445
:2047C00090947068748C887484988C7C788480788CA088747C6C6484786078A0987864600D
:2047E000748C949888747C84786C707478888880848C787084989484848C787C9C88808865
:20480000786C747C7464607C8C7C7070909478807864848C7480808088747C9C7868888828
:204820006C7898908494886C809C8C68749498706878787C8088787078747880848C8C8478
:20484000806868948C78807C7C847C7C84746C8084848884747C947C688C9C7C64688088A4
:20486000848898A088686C787C88846C74887C8490706C80888C8C78646C84907C80A49414
:204880006C60707C8C847C9880648884707C747CA088686878909074788C906C6890806094
:2048A00074A09478807064747C748094908C74688C9468749088807C7C887C7C9490786804
:2048C00074887C7C948C708088787C80747478747884888884746C74747078747488887C50
:2048E0007C8490847C808090907C7C84787888887070888080806C80947C7C8074807C74C8
:20490000808C8C888880707474687C907C708488747880787C808488847C747480848878D3
:2049200070807C7480848484949880807C7C8890807078948C706C68687C84847C70808C9F
:204940006C708C848488887064949C80748888806C6C8C88648098807884807074807074A3
:20496000888C786C8090787480808C847878747C908C8C887478888078748C947C786C744F
:204980008480847C747880807C6874888088846878988484948C8880747C7C80948870702B
:2049A0008078708080787C8C9074687C84888C88747C90786C686C888478746C7884788077
:2049C000848C948880806C6C8C908894948C8470607478709CA068708C78809084888C7893
:2049E00070687084806870888478807C646C848884909C88747C80706C8498987C6474802B
:204A00007478748098887070788890848080847864708478749498787074708890706084FE
:204A200098949884646C748C8874807C78788494888894888894746084907C7C9488646452
:204A4000706874847C8484686C747C848088846C788C786C809084706C7C9498988484849E
:204A6000889088847C707C74708C8C78747878686C847C7C88888C8C7C78747C948C707076
:204A80007880887C7070788078809084848074808480948870746C7C90747090907C747856
:204AA000686C9C9C8C80709094747C6C6480948070787C7C8080848480788C8C707C8C8006
:204AC0008484888C848074646C9490849084787868647C8C88848474606478908C7C80801A
:204AE00074747C888484806C809C88647074788888888C6C6C887C747C80909C9080807CCA
:204B00007074888C9088606078707C88948C7080947C78807C8C94806C748888746C8088CD
:204B200070748478747084948C8C7C7888886C68888C7C7C7078907C6878707494888088C1
:204B40008074808C9880687C84807C8494806C6C848C80847C7080908488888084887C7845
:204B600070788C8C8484707080786C70848C74748C80748488786C7C7C748090808094847D
:204B800070708C907C686878808C989078848C747488948880808070607C8C706884987849
:204BA000647880888884887C808C848080788C88787C786C74786C7888989870687C7C882D
:204BC00080788C84808C88746C708088806868808C88848488949488807878888C847C88B1
:204BE0007C7484746C74708084788C847C8C78687C8494906870807C7C8478748078788431
:204C00008890847C908C747C807C706C78847C78808078808878706C749490848C84707CBC
:204C200088888888786C70748490888C947C64708C8C78808870747C6C7884707884748CB4
:204C4000906C849C8874849C9870688480748888646C887C6868787C70889C847088846C8C
:204C60007890908078686C908C7C808084848480787074909880747C787C7C6C6474807C88
:204C800078746C84948080807C8C90848484847C80948068748880606C8C9088786C78803C
:204CA00084888C807C705C789C908C847064708880809C887890846464809484707C7C6834
:204CC000708C90808084847C7474848880848C8C88806C647480787C8C8C807C7C7C707008
:204CE000889C9488745C6484847C748888605C7884908C90A08C787078847C7C90987C70B8
:204D000064647C807C7C80888888887C848C88988C6C687C84807874788480646C68648027
:204D20008090A49C847C6870848C9C8064707C7C8080807C7C7874787C849C9C848484743F
:204D400078807874646490806C848C7C6864789494948C88907C8094887C70687C887C7897
:204D6000888C8084846468787C8CA0947C6878947868787C746C748C94888490846C707073
:204D8000687484809C9C7468707C9080707C847C84887C7C8C9880748C7868889880747C1F
:204DA00088907868747C808C889094786C7C7064788C84787068787C8890888C847C80782F
:204DC0007C84849094846868748878747C7C8088848484787C848C9080787C747C747898E7
:204DE000906874847C786C7C948C948C747C908C7C80947C687484807C8484787C78747CCF
:204E00007C787C788C947474847C8084787C80788C9480788080807C7478848C8C84888882
:204E20007064708C846C7480748898948C78746C6890907078909074749C9874646C8094AE
:204E4000948C8884786C70747078807C887C7488807C88787C8C80807C7C909484888C6C56
:204E600060708080788490907C68687478808080989C786C7C7C7074848878707470809CA6
:204E80009C84787C80706C849484809898706C807860688C84789490707C7C84907C7C801A
:204EA0007884887878887C70747C787C7C8488788080747C7C6468808C8C7C74808488904A
:204EC000806C7C80707C8C88848C8880806C6880887C7C848C88787888909884687C786CFA
:204EE00078848C8474788068647C8488746C8C9C9488747084808890685C7870687C888822
:204F000090907464688494948888807C847C747C808078747C787C8874788C88888C807899
:204F20008498A0807088785C68746860809C908480786C687C84788C947874848C80808CA9
:204F400088746064847C74889894847C6C7078788498947C707C887868708C886C78887CB1
:204F600084988C7C84787070789084789890747C807C6C6C80848894847468788068748865
:204F800078747C787C8088988C8078686878808C8C88886C6478887C748890787884809045
:204FA000908088988C746C7890746490946860787C747C8C908C9C90686888886C709090F5
:204FC00070606C88786C848078847C707084988C94A088646C80847068808C8478746C7065
:204FE000809088989470848C7C84888C8C74606C74747470808C84747C888870608CA080B5
:205000008090887068748488846C6C88887068909C90807074807C80908880807C807464D4
:20502000648090908C7C74989870808C786C7080847C788C8C74787C748070688498988078
:20504000809088748084747474808C888480808C807064688C9880748C94787078786C68A0
:20506000708480747C7C78848C808094906C749C948C98846C746C647484908C88887C7824
:205080006C708C807C8C887C8884849070709884686C68747878989888847C7480787C8040
:2050A00074848C78707C887C707C9080706878847C8894908480907C6C888474888C747018
:2050C0007C8074707C8088847C84787C9488748C9080787480888490906868788478747404
:2050E00078747C949478787C747C8C888480847C7C90947C6868687080888C848098987CA4
:205100007470788C847C80787C8880686880807484846C7C908C94887C807C849484808C9F
:20512000807C8C7C707470707C84888C807C88807C847C7470707488908880747068687CFB
:205140007C70748898908480806C78948C807C808C847880888480887C687494988C9488F3
:2051600060607C7C70808C847C8C90786C74706C809480687C90807488907464808C7C70C7
:205180007C90909084747C746474848C987C74847C7C7C707C7C70788490947C788C8C800F
:2051A0007474807868788C7874887C7888787488948884848880708C948074707480788033
:2051C0007C6C7C8C7C789088747C848C88787C7C78787074806C6C7C7C7C78809498946C17
:2051E0006C887070908C88887C7C7474847C7080807088988C80847C7C907C7470608090E7
:2052000080888484806C646C687C9894807888908C7870807C74747C7C7C8C94888C888892
:205220008870787C7C9C9C745C607880646C88887C84948C6C647C8C847C7C7C747C8488DA
:20524000908874646470807C88908C9090848080808C8880787C94946C647C7C787C807862
:205260007C847C7C9494847078886C60848C78686064787C80747890988484949078748C6E
:20528000987C7088908474788488706474707084888C94888088786874888878747C74686A
:2052A0007490847C847C7C8C8C84787C8C8874808C746880846C808480807C74687094940A
:2052C00090907C7C7C70848478908870707C78808880808080847C787C80807C7C788484EA
:2052E0007470748494887C807C7484948C7C7C88806C6878787C887C7884908474808474E6
:2053000070889074707C80889084787C70646C748894807C88848C807884908C80748080A5
:205320007874808870687C7C787C9094847C7C747C887C787C8088807C8C8C7068747874D9
:20534000748C988C7C80888080887C6C707C84948C808474646C7480847474788894887C65
:20536000848C88807C74707C8C88888880786C747C7478808084747C948078888480888839
:2053800080746C88906C7884787884807C7474888C847C7C807C84807C8888848474646871
:2053A0007C747C948C78747884949490847C7878788884807C6C747C787478707880848025
:2053C0007C909080848C8080807C8C846C6C7C7C8C88706C80847C8090887C807C788084C9
:2053E0008880787C7C6C788064648C94787484848C9488847C7C90846874888C847C8878CD
:205400007088848484889084807C788C8C746C6C74887C6C70787C8890806870888C7C70DC
:2054200074848C8074787C809080789894848080849088808C88686C8C908068647C786484
:20544000707478888084808490808494886C6C8084807C7C80847C7C8C7C7C847080988C44
:20546000807C8088747890746478847C787074888084908070808880888C786C7C88847478
:205480006C7C80707C807C88787C949488787C989070747C8894847C7C70707C888C807C10
:2054A0007C848074747C84806C6C8084847C787C847C80887C6870849494909088786C742C
:2054C000807C7870707C8880788094947C6C84847C7C7C807C70788C8C7C68708C988C80F0
:2054E00088948470789494746C847C6868707C6C70888478807880989880748C90786C78EC
:205500008888746C78746C70787C78808C8484888C8C9894887C6C808860607C80707C84E3
:20552000847C7C8C8888948C8C887C7C7C8088806C748888746464888C80808080888C943B
:20554000947870808078706874848078707478787C747C8078989884948C78847C6C80809F
:20556000708090747090907C74848874788C7C7C949084706478787890786C8878647C9073
:2055800084788084747088988880807070807C7C787C9488748498886C7480706C8494802B
:2055A000787C80807C8C88747C806C8094887878889078787C6C708080807870848874882F
:2055C000847C888874748088887C7C80807C6C6C888C78748080808890947C748C8C746CE3
:2055E0007878707074707490987C6C7C8C84848C78648490786C7490987C747870849888EB
:205600007474787870788C8080908C74707C8080847C707C807C8C88888470788074747CEE
:205620008480808C887C8C8874707888847484908478848474707C807C7878807878888C7E
:20564000888C7C7880847878847C706C6C7078848080888C7874888C847C8484809488786A
:205660008C8C7868748C807070788888808878748084888C706C808C90786068888C7C787E
:2056800088908874688088808C988C74788C8C80807C7470686888848488807C848070801A
:2056A00080747880948C748888746C707C84888C747490988C84808C746880707084808406
:2056C00088807C7874847C749090808080787474808C7C747C707C989080807C78787484F6
:2056E0009080809C8C647884786864788C88807C80888C7C748088787C8C80747080907CCA
:205700006468707C88847C849C988C7C847880948C747474707874787C7888847070848CCD
:2057200080787C8888808C88686C8C807C846860709088708098988084887C747C90848075
:2057400084788080707084907C6868888078808894807C84747888807C7C6C6C80848074B5
:205760006C788C94908C847C7474889088847874808084909480686C8880747880847C7C25
:20578000847C7C847C7074847870807C788C94908C787C7C7C6C68909C7C686C848C787C4D
:2057A000847C80807080947C748C9C887880806C6870748090786C84887C808490908080F5
:2057C00080686880888C8C7064707C847C8098947478847C8080848C84807C78747C786C25
:2057E00074806C60849888807C90947C80887468708490908C7C6C808464648890888078D9
:205800008490848C9484807868707C70788480888470788080848888887C748074708088A8
:2058200094806C707C7C848888806C788C8878787C808888787C807C7874888C787884888C
:205840007878848080888474746C64748C9C9874687C78787C80989884747078909484845C
:20586000746C707484888088887C7C7C7C7878848078909884787C746C748C886C687C8094
:20588000787C8890907C747C74708884787C808C78687C78789090787074808080888C9024
:2058A0008C7C7068809088808C88706C8490807C80807C787C707C9084788884848C8470F8
:2058C000707C807C74787C747080847C84887C707478606C9894807C74808C889498888000
:2058E0007C74647088848890847C80908C808490786C80787080887C706C788070686C6840
:205900007C9C94808C90807C8894847C807C6C707C787C9088787088946C6494988084883B
:20592000787C74788C8478807464706C687C9494887C848C78748C948C7C68788074747CD3
:2059400080848480847C68748C909488747C888888888C9084787874606084888090988C17
:2059600078687880788C8464707C8080809898786C7C7C6C6C849084848884807C74789073
:2059800090747C84808070648090848074687884889C94786C7C8C846C70889894847C7813
:2059A0007C7C6C8098887C8878747C7C8C80707470787868708C9C987C747474707C80903F
:2059C000907470807C70748490907064849074708C9494787C847474807C7C8080788484F7
:2059E000706C849498887474706C8098908884747C8C7868788C8C7C8488747484888C80A7
:205A00007478747C806C7C9884748084786464809488888C786C7C7C70848C888080908CBE
:205A20006C74949884787C7C747478888C80786C68747C8894947C7C8C887C70788078849A
:205A4000846C74847C8484747C7C7080787088888494887C80747C8078847C706C748088AA
:205A6000948C808090948070686C889894746C6C7888807C80746C686C74808C94948C803A
:205A8000747C8C887C849484708488747C8078888078887C7074748090888074747868705A
:205AA000989480706C70707078888C9898806C707C80948C7C786C7C8880849090807C70E6
:205AC00068747880888890948474747C746C80888084888880748C8C74788078706C74801A
:205AE0007C80808484788080809488788C947C6C6C808C888C7C74787078848C80788078B2
:205B0000707C8884807C7474787C707080847C7874808C8C889088788888808488807C8899
:205B20008C8074787C7C747078808480787C7C7C8484807C6C6C787074849098846C787CE1
:205B40007C8084908C7C7878848C807884847C7C80746C7C8C8880847870747884807C8469
:205B600078707C8074849088847870889480707888908080847C787C74708894887C706C55
:205B8000707C90947C70787C7C7C8488847C70686C787C808C8C7C74787884848498987431
:205BA000687880908C7874746C78806C808884908C80808474707C8080808888787C807435
:205BC000707C7878706878807C9C98807C848074707C8884808484807470748494847C780D
:205BE00078807C8894908480746C7C80787478848474706C64788C8C908C7C8084888C78CD
:205C0000708C88809480646C9498807878746C6880887C9094786C7C7C6C748C84788480C8
:205C2000786C74909888707080807C8488888C8488948C7868788C7C708080787C78708880
:205C400094807C807870707C88848890847470747C9090746C74848470748C847884948C58
:205C6000746C84908C8074808C7C74808C8C887874808878707880847C7C80746C80908C48
:205C80007C6C70908064788C8C888480847C647488888C80707880849C9C8478747C847420
:205CA0006C788088887C7C74646C8488807878848C8488848090887878847C646C889C8814
:205CC0006C80887C80807480909494848084747090987470807460647C9090746474888800
:205CE000807C848C88847C8C84607094847C7C647894807C84747C888C947C78948C787C90
:205D00008C80747870646C80887474909478788C8884888C84787C848884847C64688C88B3
:205D20006C748C84788894887C8480848078747874747C849890646888806C7884847870B7
:205D4000848C88887C6C6C787C7C80847C84907C7C8C989074708088949080706878807C43
:205D6000848088907C78887C848470787C747C7C787C8C90847868687C908888888090980F
:205D800080748484746C70746880987C687080887C707874809084808C8C8C847074787C7B
:205DA00088847478808078848C8880808C8870707C8484888878707880807884806C6C7827
:205DC000848484847C7C888C808888786C7C7C6C787C74807C747880848484888074848CE7
:205DE0008088887C80787474808C887C70707C80848C8074808C8074808080786C748088E7
:205E0000808094907068788C9084748084808480808C8468708078808880807C70808874A2
:205E20006C6C78887068788088807484947C78808C8474889080807C8084848478748C8096
:205E400068789898787480747C94908078746C8084747470707C6C688C948878787C88849E
:205E60007C84807C7C7874808C8C8074706C7088887078888C8C7C7C8C847C746C7C888066
:205E80007C8888807C807C7068748484787C84909884788C887874708488707C8C7C747832
:205EA0008080707484888884787C9498886C6880907874887470848C7870787880847C702A
:205EC0006C84948C807C74707C848880848C8C887C747C808070789094887C7C908C7878A2
:205EE0007C70747C747C7868788C90806C68847C6C8C9490847C808478808C847C7C7C80F2
:205F00008084847C808C8470708480787C808080808080786C789084888874747C788490A5
:205F200084807C848C7C7884788088706C7C84887C749090787C807C8884747C8890887069
:205F40006C74788C9C886C748888808494846C7884786478847478747880848874748C987D
:205F600098887878747480848480848478786C688C9478707474848C80909880808070704D
:205F80007C6C7090907C707C88787884848080848C8888847080908074787060607C909C39
:205FA00084687888807C849088808080807C7C848C88806C6C78808C807C8C887078807CFD
:205FC000808084807C7C808C746C70887C78847C7C888484888484848078787074989894B5
:205FE000807070787474847C78847C8088847C808480786C6C7470789494907C7078787825
:20600000848C8888887C787C7C7C7C8084706C7C88948C78808078848478706C7C8C908488
:206020007474706064809C987C808C807C847C848C7C706C747C80809498705C7080787CD8
:206040009894889C9C847880786C808C70707C78786C78908478706C7C807884908C847C3C
:2060600078746C687488908474707C8480848490988C88948C687498987068807864687C64
:20608000888084745C6C8C8C787C9490788888686890988080807074849494746884908404
:2060A000807870849084787C7C74787870808480847C6C6C787C8080808490806C788C9038
:2060C0008C8078807874888888887C807C74787880949470788478848074849080707C84CC
:2060E000787C8888847C7C8874646C9094847C7C7C807C78848C7C788480847C74808480C4
:206100008080787074707484949088808080747888888884807C6C68889480807C707C7CB7
:20612000788088847C78808880747080949084888C7C6C70747C7C78848470809490907C5B
:2061400064748470686C90A0846C7C78686C78807878808C908888848C9C88686C787880AB
:206160008898988078786C686C70849078788C887C707890908470787C7478788494886857
:20618000687C88887C8C9C84888C7464647084848C84707C80686484907C7478808078845B
:2061A00094908C807878706C6C7C989480808884746C7880808074707878808C908C8474F7
:2061C00074807C7890988C887074908074747C948C707074787C7C848C7C78807C808478E3
:2061E0007C8C8C7C70708088807880888880787874788C908480808C806C688890746C64E7
:20620000646C80807C888C808484809090808C94848084846C647C908C807870787480947A
:206220007C788C848484747884909878646C68687C88887C74747C7C7C84808C98908C7C7E
:206240006C788080887C6060748078748CA0947C808080847874909C9484786870807C7486
:20626000787478847C80807C888C88806C74847C78889088847C746868848C848488888836
:20628000887070808C90746C74787C94947068787470707480807C88909088747078848C5A
:2062A0008878708094948C88847C747C887C7484948C887878746C80886C748888848484CA
:2062C0008480807C706874807C7884908478787C7474888074888C8490947C6C78848484EE
:2062E00080807868748C8C8468608490787C9898888C9080706870788890787488908878AE
:206300006C7C806C7C8C7C7C808494948880746C60608094847880847C7C787884908C88B1
:206320008480888C7C809480707C847468707C7C7C787880787480889094907C8880708871
:2063400090786C748488847C847C74807C7C8484747C90887C7870707C847C706C748088A5
:20636000887C747C908C80848C887C809090888074706C708884747C7C747C78747C849429
:2063800098806C807C6C7884808084807470848478909C78687C8074747C8C94846C687851
:2063A00090787080848C8880847C8090908078787C747C88808488807C7474847870888CD9
:2063C0007C88908074686C84807884747880707C8C8C908C8478707494988C80807C807CC5
:2063E00064687470746C78888C908C7C808C8C887C7C80747890887070787060747C7C9029
:20640000989488807484948074787C807C787C807C7474706C70707088989488908C7C847C
:20642000807C848078807C6C748484786C686C787C84889C9C807C8880706C7880787C84C0
:2064400080787478746C808C808C9C807080888C908470687070748490948C808070606498
:206460007C90989884788884707890907C6C68808C7470889890787470686C78787C8C8434
:206480007C847C6C6C808C80788484807878807C848C888484786C8094807C8884888C80FC
:2064A000808884888C7C7C8068646C747C7C84887470849084889488747880808880707020
:2064C0007480846C70847C747C88948878807C748888808C80686C8084808088846868900C
:2064E0009880788094987470949488887C7470707470707C7C78808080888084908074849C
:206500008478787884908C807C7C7878747480887C7C807C7878808C706C7C8088807878D7
:2065200084948C84847C7C7070889898907C746C7088907C748894846C789080707C787053
:206540007874687C888084848884707484847884988884948C7474807C74848C74747C785F
:20656000787C787C8080848C7C7C909480708078687C806C6C809494888484787C8078744B
:20658000849090807C7C80807C74787C7C78747C888880848078706C7C8C7C708498907817
:2065A00070847864748C8074808C908470708490886C6C8890887C7C908C7078887C74741B
:2065C000787C8490988C746C706C889C9070809088888C8474707C7C6C64708480707484F7
:2065E00088847C64688090948C88909480687884807C787C8474708C8478848C94886C7C93
:206600008C7C7C8084887C68686C748088807C84807480847C78909C908488847C80787496
:206620007860606C7C80807478908C808C88807C748C9C8C70788488806C7088907C7074B2
:206640009098807C8080807C747C887868707C706478908878748C8C787C8480848888786A
:206660007888807898947068687C847C7C8C80788C9488787474747888887C8080707C903E
:20668000847880909484788488807C7C847C6C6868788C887880847C84807880888C888CF6
:2066A00094846C6C7C807474808074787880909084847C7078747C88787894947060687C52
:2066C0008070747C889494807884989C8C847C68748C8C847C787C6C6478807480807494C2
:2066E00098847C84807880887C64647C80787078848490846464889894888084786C747CE6
:206700007C8090906C6C84908C88808084787478808C8C80848474747C7C847C70808C8475
:206720007C7C74787C708088707480808C88808C8C7C6C7080808488909488706C706C6CBD
:20674000788880748078788888848884888C7C6C74808888787068687C8074809090908855
:2067600084888888908C80888C7874706874888080807C8478748890888C8C846C60647C39
:20678000888C7C646C807064808C88887070848084908898A08478847C7C78788874648029
:2067A0008C8880808C8C84848078787C7474808C8C807470686884949084807C78808884D9
:2067C0008488847C78787468788C80788C8878747C88948874808C80747488948C706C6CED
:2067E0007C8484847C8080708090887C74747C786C7C887874808884707890847C88908CB1
:20680000908C8088887068788884787478746868788494907470809090908C806C647488BC
:2068200074688494948C84807C7C7C74788C8C88948C74707070707884787480807C808088
:20684000888C7C707C7C7C8C98908C989070686878887874887C707C84807C7C7474849048
:2068600078748C908C8878747C7C8084807C8488808078747C7474848494987C70788C9404
:20688000806C747C7C84887C7070849488707080888C8C807C788088807878786C6C746C7C
:2068A0007078848874809888849484849480687C909090847878746C787C6C6C7C848888D8
:2068C000948C78788488888888806C70807C88846C687084908470849C9C847064748C8CB4
:2068E000848478687488846C68748478808C8884848480888078746C7484847C80888078F4
:206900008488786C748C94908078848C8C887C8088848884747480787C88888474747C805F
:2069200084846C68747C6C707C80807C7474848C846C789898847888887874807C6C748CC7
:20694000908880809090889084748088807C848068647480746478989080807C787474844F
:206960008C847C6C6484907C80846C687070848C7C8898989088888070708088847C6C7843
:20698000907C68646C848470788470788884989470687C8080888478787C8C90807884902B
:2069A0009090847C8078708490887C747470687080888C84706C7884808084807468747C47
:2069C0007C888C848478809088807C686C908C848C746870788C8C787C8C84747C808080C3
:2069E0008C88747088907C749094786C6C686870908C6C748C94947C6C7C7C8894787088C7
:206A00008878787C747074707480808C949898847C84847C78687C9888646470747C7C78DA
:206A20008488847468708CA0988C888068607C948884807870707878788C94948888847C3A
:206A4000847C7C847478806C687070787C787C889080706C809090908C8070708080808896
:206A6000887C7070707C8C8C90948C806C64787C707C90887870749098806C748880788052
:206A800080848884908C88806468807874908C7C747084847480908C7C78706C7888848022
:206AA0009080647894908474748C947C6C7478848C90908470687C807870788C8C6C6C8C02
:206AC0009484787C8C8C847C7C78787474848C8078807874746C7C948C7C70748884809CC6
:206AE0009C7864687470788C8C7C808884807C787C90908484848C94847C84807470686CC2
:206B0000807C707880808074747C74748C94846C6C888C80848078808884848880747C88A9
:206B200088706C8488848C88888C786C7084846C70848C806868787C7C8088847C80949481
:206B4000848484888C847870787C74788C88706C748890807C8C8C807C7888907070848049
:206B6000848870646C6C747C787C7C7C9498847C80807C707C7C747C88888C847478808471
:206B80008C7C80908480949898886464788C7C707C786C7C887870747C84847C78809094F9
:206BA0007C6C788484787C8C847C88908C8C7468747C88948880847C7074888870687C8005
:206BC00078909074788884887C7074787C80787C90887880807478807C7C8C94887C8080BD
:206BE00078809894786C747C7C70707C88909480747C78849080788C84706C7074808884C9
:206C0000807470787C8C908C9484747C8884908C7874808480706C7C807070808484847C94
:206C2000808C80787C848074788888848890806C6C78706894988880807074808488847078
:206C400074746C7C8C84809090806C687C949084847C8088787074787C848088846C6C7C80
:206C600080848C8478746C707C7C78788084807C8084989C88848C7C7C786C80847884881C
:206C800070646874807C809490746C8490949084888470686C78888880787474747C8C8C48
:206CA00084808490907C6C70787C848080847C645C6C78849C948C84748098949494887CA8
:206CC00060606C80787C80888868647C787C90848090947C74848C8480908064647880704C
:206CE0007490948C7C74747C8884808C8874707880847C7C88806C707C7C80847C88948898
:206D0000807870788488908C786C686C787C8C907C6C70788C8C7C7C8080747074787880FB
:206D2000949488807870707C888C8894947C74848074848874747470807C70889894847037
:206D40006C787470809088787068687884888478707C84807C80848C948C707884787C7CA3
:206D60007C807C7C84786C748890908C7C748890746874908C70707C787C88787C8080804F
:206D80007C7484908488948C7C74787878808C846C707C84807C849088706464707C788C3F
:206DA00098847474809088788080747C848C8878747C888C7C74788084787C9494887C7CB3
:206DC000807C747C84887C687088806C7C94907C7884788094907878807C7C7C7870747C03
:206DE0007468687C887C748090948C8084908C806C74908070808C80747C8C8878788088A3
:206E00008C88888884888C747480747488806C646C787C74788C8C90947C80908078808082
:206E2000746C78948C7878786868707C888C8C8C8C90948884848074747470787C7484987A
:206E40008C7474808070708C988474748494806864708088807C807C78849098988C8C9412
:206E60007468848C80746C707068787C84988C70808878787C88806878948C7C706C7884A2
:206E8000887C747C80808888949C908C8C7C6C6C7C807C7874706C74809094887C787884F2
:206EA000887C84949080807C6C686C787C7C8888787880849898848C8C786C687490887CD6
:206EC000848078786C6C809088808888847C6C7484848888847C6C6C8080808C8474747CFA
:206EE000808088989C9880686874787C90908074747874748498806C787C7C8880707C8CA6
:206F0000908874686C708090887C8084807C80887C8094906C64707C708094908480847499
:206F20007088948C848080847874786C809880686C70788088949884808484807C74889045
:206F400080706C686C74747C888474747C848488908884888884806C607088848074646CE1
:206F600078788CA0A0A084747C7C74889C947C646C74707C88847C746470888C8C8C8C8CD9
:206F8000807C888464606C7C84746C78888C7C7C90948070787C787074889C90787C7C6865
:206FA000747C7C888C807878809090949C88687480746C7C8C948C80746878847478908CC5
:206FC00078707880787080988868687480788088807C84888C88807C8088909484747064F5
:206FE0006078949894887880807078847C7C787084847888908078746C6C747484909084C1
:207000008490908478788C8C787888807C74687C949084787C887464788C84747C8C7C6890
:2070200068788C9080746C68707878888C808890807C807C848C84848084807C7C8888885C
:2070400084807C74707C7C70787C8480706C7C84888C787884807C7C808880788888706CA4
:20706000747C7874808C948C7C748094948878747C8078787874787C74747070848C808058
:207080008888888C90807C88847C74747874706C687C94908480707C98948C909090806CBC
:2070A00078786C787468787C6C6C8084787C888C7C7C88887C747C8080807C7464687C78A4
:2070C00080948C8088888C90807C888C887C7474787C847C646874747880808894948C8884
:2070E000786870888C7C707C887C787C7C7878746874909080848C8488887C70686C78880C
:20710000847474808C887880988878848C90886C70808080848478687084848484746C7C97
:207120007C80888C8C8C847C70686C74807C707080989C8C8480746C789094807C786C747F
:207140008C9080707070707C787C88989C8C808C90888C80747064647478807C7C888C883F
:207160008484888068688C94887C748088888884706874787C80807C8C908C8C8C8474681F
:2071800074848480746C8088807C7C7C88907C6C78808494907C7074888C80808880807407
:2071A00068748088887C808C7874847C747874788078789094907C708C9C8C807870707407
:2071C000788490786468787C88909084748890807C84848C887874706C70747C807C7C80FB
:2071E0008C9090807C8C847C84807870748488807C7C74787C6C687C909C94888C7C70847B
:2072000090847C7C7C78706C747878787474849490848894A49C88806C5C7C98907C7C805A
:207220007464647C887C80807C888880849084707884806C68788084888088948C7C7070A6
:20724000889C9C9C8068707884847C747C80746C6C7C88847C78808070747C8488848C8C3E
:2072600078747C808480748490908878788C908C848078706C6C78807478847C7074849446
:20728000908480908C74687074788480787C7C7C8080889490848074788488888C948C70CA
:2072A000646C7874787C747C908870748894887C808074707C887464789494806C68747872
:2072C0007880848C9484747C8C909098846C646478887C7C90947C6870848C7C78808478B2
:2072E0006C6C7C88908C8880786C68787C747C8C90887874808080888084886C60708090EE
:20730000949098906864707C7C787888846C68788488888C8C888078707084888490948461
:2073200074747874788078787464708C94847C8C907C7878787C707084847C807C74786CF5
:2073400074888C88807484948C909C908880747468687C8C8070606480948C74748C8C7439
:207360006C849488807C7870707474707078808C88787C8C8C8C8880849494887C747C8019
:2073800078807C6C6C80808088848C907C74787C80847C7C888C807C7870707484847C7C3D
:2073A000848878788C8878787C7C787C848888887C70708088787C84808084847874748001
:2073C000807C80848484807C848C847C78787C7C7C80807C80887C70788888888C84707CB9
:2073E0009090847C788080787878809080707074787C80787884847C80848C9080747878BD
:2074000080888480787080888488848488847C8480848C847C888C88847C786C6874888458
:207420007C80807C7470849080747C7C787C8088847C84847C7C7468688088848C8C847890
:20744000748094909090807C786C788C908C7C7C8880706C7C887C687488807C8480809024
:207460009080808074686880888C9C9C74646C78848C80808880787C8C9898848484706C00
:2074800078847C686874787474808C949084888C847C74748084888C8884807070746C7448
:2074A0008080847C7888989894848484786468747C8084847C746C646C78849088808084FC
:2074C0008C94908C8880787470707C8C8C807C84787480888C8C88848070707878747880B4
:2074E00080787070787C88847C807C7C807C848888949480746864687898A08C88785C64E4
:2075000084948C7C74747070788090908C8C847870707C8884849090887C686C787C84906B
:207520008C7C7064647C80809090846C648090909084888878746C68748084888078787CAB
:2075400084887C808C88787470748488887C7074706C748C94949080707488908C80788433
:207560008484887468707C78746C68707C807C7C8C9084808C8478808894988C8068646C6F
:20758000807C909478707C84807C8084847C7C747480847C787C7874707C84807C88908417
:2075A00078787C787880908C8C907C7480807C84807C74687480807C787C88887870787823
:2075C0007890988C706878848084847C7C7C74706C70748090908C807C7C7C8490908474BF
:2075E00070747880787C8C8C807864647C8474889884788C98887870848C807C746C6C6CFB
:20760000748C989888746C7074808C8C80787C8088887C78807C6C6C8080747C8C90847882
:207620008490847474787C80808C94807474707C887C6874807478807C8488888C84808C6A
:207640008C8080786C748484787480847C8088908C746C7470748C9884808890887C6C685E
:207660006C78848088948C7878787C807C7880807C8494948474809480686874809488701E
:207680007884848078747C84888C88807C8080787C8884787C807478848078707880787832
:2076A0008C9088848C847C848080847C7C7C808478707C847C7C8884808488847478807CB2
:2076C0007078747480807C787C8480787C8478848C848478707C88888C908478788C9084BA
:2076E0007C7C7C78807874808474707878787C74787C809094887C78748090888484807CCE
:20770000787474788890847C7C7478888C8480888C78686C7C747C84808880706C6C7488DD
:20772000909094908C8480847C788894806868686C748080787878788090908C8C94947C0D
:2077400078847C6C748C8C9088706C74747C84888888807C7C7C808880787C786C7C887C71
:207760007C847C70646478888C90949890888C84746C788088786C6C74848C807880807C3D
:2077800080888884888C8C847C7870788484848C7C6C78787C7C6C7C9090887C787C747009
:2077A0007880888078787C849090887C6C74807C787C84888C846C68807C707C8C806C7421
:2077C00084908C848C94847470747C786C74889488746C848C808484889080787C74809485
:2077E00094907C605C64707C848C908470789098887878808078706864707C848C84747019
:20780000747C8088889094847C808484808894948078747070747884847C7C8078706C7888
:207820008C8C84806C6C808484888884746C70686C88949098947C74787C7C888C7C68687C
:207840008088848484746C74848880747480949484808884747C8C908880787474787C7834
:2078600070747884807874707C8C8C747080848488888078808C786C7884889084787C7C4C
:20788000746C78888C8C8884807C7884887C7C7C7C78747078888C8074707884847C8C9010
:2078A0008888848080746874808484807C7464748480808C90847C7C848C888484807870F0
:2078C0006868808C847C78747080908C7C787C84887C78787C888880848C887878747080F4
:2078E000949088786C78847884908C847870747C80888480807C7C7C7070848C84847C6CA8
:207900006C787C787C9094847074808C847884887C78788080707080807C787C808C948493
:20792000808C88807C787468647488889090848080787884908C7C7C888884888C80746C47
:20794000787C787C7C7C78707480807C7C7468748C888888807870788890807C8478788097
:207960008C908070808C808494948C7C70747C78747878888C8484808080808878707084FF
:207980008C8C88787C888884787C847C747878788080807C7C7C84847870707C807C78802B
:2079A00088888C887C848C7C787878808C8080847870788480787C84787890949484808893
:2079C00080707C7C7074746C74787C8480808880808C8C888C84807870808C7C706868683F
:2079E00078848480848484909494948C848480747478746C6C7C8C8478747C7C848484846F
:207A0000848C847874708088888C78687078707480888880808884889090949480787C7856
:207A2000746C707C80747078807C70788C8C8C8C8070707C888C88746C7080908C84807CA6
:207A4000808C88787C807C80848C8C84746C6C6C8088787C8C807C7C7C807C80888480784E
:207A60008090948878707478786C749090847C808880788084847C7474807C7078887C7446
:207A80007884908C7C7880889490807C6C647488847878746C6C747C889094908488847CEE
:207AA00080888C7C6C74807C7470788078747C808080848C908C8C8478706C6C7C8C84701E
:207AC000707C7C78707C8C887C8C9080807C7C888480848078706C80887C78808C886C6CEA
:207AE0008C98989484786C687484848074707C80747480887C7070747474787C8890847CD6
:207B00008C907C70788088909494806C6C7480808084807C78747C8C8C847C847C74787875
:207B20007C888480847874787C84887878807C747074808080888C847C7874787C787878AD
:207B400078807880908C84888884808078707888908C8478686C80887C707C8478686C7875
:207B6000808C98947C80888488888884808484706C84908C8078746C707070808C847C78F9
:207B8000807C74746C6C70788888807878808C84808C8C807C7C808C908C84787478747429
:207BA000848880807C787878848C848080787884847C787C888C84808078788088887C74D1
:207BC000706C787870748C8C807C807C848C8484808088847874747880808080807C787401
:207BE0007888909084746C7C888C8C80787878747878747C808080888C8484888884808079
:207C00008484808080707074707C8C807070788484888C847878808084847C807C70707CCC
:207C2000888C847C808080808488807074888C7C78848C8480807C78807C74808880807C3C
:207C4000748488847C8080787C888880788088807C8080807C78788080807C7C7C7C787858
:207C60007880807C7C80848084847C807C80847C7C7C7C888C80888C7C747C848074788810
:207C8000848490887874707080887C70707478787C848884807C7C8490887C7C7C7C747C30
:207CA000847C787C80807878888478788888848C8C84847870788080786C747C7478848C00
:207CC00088807C88847C7880888C807880847470747878747478848884888C8C88848078B4
:207CE00074707C84807C80808084807C848C8C8478708088807C84807880807474788480B8
:207D000074808478787C7C8084888480807C747C848880808488807C808488807C78787883
:207D2000787C807878788088807474787C8484848480787C848888847C8078748088848073
:207D40008488807C7874747C88887C7C80807C80848080847C78787C80847C7C7C8084804F
:207D60007C80888484848078787878787C808C8474747884848484888480848080847C800F
:207D800088847C78787878787C807C7C7874808884848884807878807878848888807C7C1B
:207DA000848488888080847C80847C7C7C7C807C74747C7C787C80808080787478787C840B
:207DC00088887C787C7C8488888480787C8080848484807C7880807C7C80848484807C7C9F
:207DE0007C808084847C7C807C7C7C787C8084807C7C7C7C84848480787C807C7C808080B3
:207E0000807C7C7C7C787C80848480787C84807C80807C7C787884807C8484847C787C7CA2
:207E200080808080807C787C848480808480807C7C7C7C7C848888847C78747C807C78806A
:207E400084807C84807C8084847C7C7878787C848484807878787C808484847C7C8080804A
:207E60007C80848480808080807C787C7C808080807C787C8484807C7878787C808484842E
:207E8000808080807C80807C7C8080807C80808080807C7C7C807C7C808080807C7C7C7C16
:207EA0007C7C8080807C807C7C80808080807C807C7C7C7C80807C7C7C7C808080808080FA
:207EC0007C7C80807C80808080848078787C808084847C7C7C80808080807C7C7C7C7C7CDA
:207EE00080807C7C8080807C7C7C808080807C80807C7C808080808080807C8080807C7CAE
:207F00007C807C7C808080807C7C7C807C80808080808080807C7C80807C80807C7C808091
:207F20008080808080808080808080807C7C807C7C7C8080807C7C807C7C80808080808065
:207F4000808080808080807C808080807C808080808080807C7C807C7C7C80807C7C7C8049
:207F6000808080808080808080808080808080808080808080808080808080808080808001
:207F80008080808080808080808080808080808080808080808080808080808080808080E1
:207FA00080808080808080808080808080808080808080808080807C7C808080807C8080CD
:207FC0008080808080808080808080808080808080808080808080808080808080808080A1
:207FE000808080808080808080808080808080808080808080808080808080808080808081
:00000001FF
